:1000000018308A002F2C0000FF00030E8301A1008E
:100010000A08A0008A010408A2007708A300780853
:10002000A4007908A5007A08A6007B08A70083131E
:1000300083128C308400001C1F280C1832282208E0
:1000400084002308F7002408F8002508F900260892
:10005000FA002708FB0020088A00210E8300FF0E0B
:100060007F0E09008A110A1241280A108A100A110B
:10007000820700340034103430348A3400340034C1
:100080002D34061D452806114628061564000C105F
:100090008A110A121F28871087160530F700F70B00
:1000A0004F280000000000348C1A5828640054289F
:1000B0008C1E58281A088316B9008312981C6628CB
:1000C0001A088316B90083121812181683163908F5
:1000D000F800831200342908073C031D74280730F8
:1000E0000C1E70289900B32805308316A700270836
:1000F000063C0319B2282708053C031DAC2829300B
:10010000A90083126F088316A600043083120C1E08
:10011000872899006F080C1E8B2899008316A80168
:1001200083126F08831628020318A6282908840062
:100130000008AA0083120C1E9B2899008316290828
:1001400084000008A606A90AA80A90282608831297
:100150000C1EA82899008316831254207808831651
:10016000A7007728831200349030A9000130AA003C
:100170002730AB00831681138312861DC2280230FC
:10018000AC00C4280130AC000430EF006B20003418
:10019000C830840000080319DC280130F800F7019A
:1001A000F70BD028F80BCF283030F700F70BD62804
:1001B00000000000800BCD2800349130A9000230EF
:1001C000EF006B202A08F700F7080319F828013020
:1001D00077020319FE28023077020319042903303D
:1001E000770203190A290630770203191029172903
:1001F00005308316990022309800192902308316A1
:10020000990022309800192905308316990026306C
:100210009800192900308316990022309800192976
:10022000013083169900263098001929831283160D
:1002300019290230C8008312C8208A150A12FC2E20
:10024000F701F80183163A0803103B18F707F70C7B
:10025000F80CBB18F707F70CF80C3B19F707F70C6D
:10026000F80CBB19F707F70CF80C3B1AF707F70C5B
:10027000F80CBB1AF707F70CF80C3B1BF707F70C49
:10028000F80CBB1BF707F70CF80C83120034923004
:10029000A9006F08413C031964290130AA00FE013E
:1002A0007E083F3C031C632902307E07293E840000
:1002B0007E088316BA000530BB008312202178081F
:1002C0008000FE0A50299C29FE017E083F3C031C49
:1002D000802901307E07293E840000088316A10092
:1002E0007E08BA000530BB008312202178088316EF
:1002F000210203197D2983128029FE0A83126529B0
:100300007E083F3C031C8629013087290030AA0063
:10031000FE017E083F3C031C9C2902307E07293EDB
:1003200084007E088316BA000530BB0083122021AA
:1003300078088000FE0A89294230EF006B208A1578
:100340000A12042F9530A9000508AA000608AB0080
:100350000708AC00053083169F0083121F08383948
:10036000C1389F000030F8001F08C73978049F008B
:100370001E30F700F70BBA2900001F151F19BE2900
:100380001E08AD000830F8001F08C73978049F0028
:100390001E30F700F70BCA2900001F151F19CE29C0
:1003A0001E08AE000630EF006B2000346F08073CDB
:1003B000031DED292A088316850083122B08831656
:1003C000860083122C088316870083122D0885006F
:1003D0002E0886002F088700A2218A150A120C2FEA
:1003E0002A088316A0002B30A100FE0102308312E0
:1003F0006F027E0203182A2A83162008A00AA20090
:100400002108A10A84000008A30022088312031710
:100410008D008F01831603132308831203178C00AA
:1004200083168C130C15831203130B08F7008B1320
:100430008316031755308D00AA308D008C148C184C
:100440001F2A0C117708831203138B04FE0A8316EC
:10045000F62983120730A9000130EF006B208A15BE
:100460000A121C2F2A088316A0002B30A100831229
:100470002B08EF00FE016F087E020318532A831633
:100480002108A10A84002008A00AA30083120317F0
:100490008D008F0183168C130C1483120C088000BE
:1004A000FE0A03133B2AE330A9000230EF076B205A
:1004B0008A150A12242FE530A9000130AA00023063
:1004C000EF006B208A150A122C2FE730A900463066
:1004D000AA000230EF006B208A150A12342F87120F
:1004E000003480308316870581308704D930860533
:1004F0000616DB3085051B30850405158516861428
:100500008312871107124B206F2287140530F700E2
:10051000F70B882A000000004B206F22871405305B
:10052000F700F70B912A000000002808FF3E03188F
:10053000AC2A013EAD2A83164608C700F501F40136
:100540004708F6001F3C031DAA2A6430C800831226
:10055000C82083168312AC2A00340A108A140A11A8
:1005600082079B2A2A08FE007E08E039A8007E0840
:100570008316C600831271220730A9000130EF00F4
:100580006B208A150A123C2F7E102A080139003A86
:100590000319CE2A6F08023C03197E1400307E181E
:1005A00001308316A000A10083124B2007110C30EC
:1005B00097000030F800043892001530831692003E
:1005C000A1080319EB2A0B30831295001708CF39C5
:1005D0009700F12A83160630831295001708CF3949
:1005E00097004B2004308316A000AF30C800831260
:1005F000C8208316A00BF52A07308312A90001300A
:10060000EF006B208A150A12442F071197019701FA
:100610004B200730A9000130EF006B208A150A1229
:100620004C2F76081F3C031D3A2B8316CB014B0839
:10063000053C031C382B8312871503108316C90C45
:100640000318262B83120712282B831683120716F2
:100650000530F700F70B2A2B00000000871105304A
:10066000F700F70B312B000000008316CB0A172B85
:100670006F2C831283164908E03E03186F2C203E2E
:100680008312712C0712871587110712871587119E
:10069000071287158711071287158711071287150B
:1006A000871107128715871183166F2C0716871578
:1006B00087110712871587110712871587110712EF
:1006C000871587110712871587110712871587115C
:1006D00083166F2C07128715871107168715871148
:1006E00007128715871107128715871107128715BB
:1006F000871107128715871183166F2C0716871528
:10070000871107168715871107128715871107129A
:10071000871587110712871587110712871587110B
:1007200083166F2C071287158711071287158711FB
:100730000716871587110712871587110712871566
:10074000871107128715871183166F2C07168715D7
:10075000871107128715871107168715871107124A
:1007600087158711071287158711071287158711BB
:1007700083166F2C071287158711071687158711A7
:100780000716871587110712871587110712871516
:10079000871107128715871183166F2C0716871587
:1007A00087110716871587110716871587110712F6
:1007B000871587110712871587110712871587116B
:1007C00083166F2C0712871587110712871587115B
:1007D00007128715871107168715871107128715C6
:1007E000871107128715871183166F2C0716871537
:1007F00087110712871587110712871587110716AA
:10080000871587110712871587110712871587111A
:1008100083166F2C07168715871107168715871102
:100820000712871587110716871587110712871575
:10083000871107128715871183166F2C07128715EA
:100840008711071687158711071687158711071651
:1008500087158711071287158711071287158711CA
:1008600083166F2C071687158711071687158711B2
:100870000716871587110712871587110716871521
:10088000871107128715871183166F2C071287159A
:100890008711071287158711071287158711071609
:1008A0008715871107168715871107128715871176
:1008B00083166F2C07168715871107168715871162
:1008C00007168715871107168715871107168715CD
:1008D000871107128715871183166F2C83168312D1
:1008E00000340A108A100A158207422B562B6A2BF5
:1008F0007E2B922BA62BBA2BCE2BE22BF62B6E2C1B
:100900000A2C6E2C6E2C1E2C6E2C6E2C6E2C6E2CCB
:100910006E2C6E2C6E2C6E2C322C462C6E2C6E2C6B
:100920006E2C6E2C6E2C6E2C5A2C76081F3C031DE0
:10093000DD2C871507160530F700F70B9D2C0000FE
:10094000000087110530F700F70BA42C0000000011
:100950008316CB014B080D3C031CCC2C831287154E
:1009600003108316CA0CC90C0318BA2C8312071281
:10097000BC2C8316831207160530F700F70BBE2C2C
:100980000000000087110530F700F70BC52C0000B0
:1009900000008316CB0AAA2C831287150716053090
:1009A000F700F70BD12C0000000087110530F7008D
:1009B000F70BD82C00000000FC2C871507168711B8
:1009C0008316CB014B080D3C031CF82C83128715B2
:1009D00003108316CA0CC90C0318F22C83120712D9
:1009E000F42C83168312071687118316CB0AE22C88
:1009F00083128715071687110000003483164608F6
:100A0000C9008312112383164808CA004708C90089
:100A1000831295240034831645087502031C162D95
:100A2000031D1E2D74084402031C1E2D45081F3C87
:100A30000318332D75081F3C031C332D45081F3C3C
:100A4000031C282D7608C60083127122322D8316CE
:100A5000C6013F30C800FF30C7008312FE2420309B
:100A6000F500F401831675084502031C462D031D8D
:100A70003D2D440874020318462D0630C900831228
:100A80001123F40A0319F50A8316332D8312003457
:100A900083163A08C9008312112383163B08C80045
:100AA0008312C8208316BC0803195B2D3C08C900BB
:100AB00083121123831601307407BD007508BE0030
:100AC0000318BE0A3E08C5003D08C40083120B256A
:100AD000003483162108FD3E03188A2D033E83123D
:100AE000A32D09308316A1002030C500C401831254
:100AF0000B2583168A2D0B308316A1008A2D1F30FB
:100B00008316A1002030C500C40183120B25831673
:100B10008A2D83162108C900831211238316210808
:100B20001F3C03199C2D0830BA000430BB00BC01E7
:100B300083124825A02D83160430C8008312C820D4
:100B40008A150A12A82B0A148A100A158207712D19
:100B50007B2D7F2D83162108FD3E0318D82D033EE3
:100B60008312DC2D8316C901831211233F308316B3
:100B7000CA00FF30C9008312952409308316C900CA
:100B80008312112306308316C8008312C8208316EF
:100B9000A1080319D82D0B308316C9008312112325
:100BA00006308316C8008312C8208316D82D8316FA
:100BB00083128A150A12382C0A148A100A15820721
:100BC000B22DCB2DB22D83164208C90083121123FA
:100BD000831607164308C40076081F3C031D162E13
:100BE000C50145080F3C031C152E83128715000014
:100BF000071AFC2D0310FD2D0314831644088400EE
:100C0000840A800C8403800C0530F700F70B062E55
:100C100000000000831287110530F700F70B0E2E3D
:100C2000000000008316C50AF12D2F2EC5014508CE
:100C30000F3C031C2F2E831287150000071A222E4B
:100C40000310232E0314831644088400840A800CA6
:100C50008403800C831287118316C50A172E44085B
:100C60008400013084070310800C8403800C440846
:100C700084000008F700840A00083F39FA0077086A
:100C800084038000840A7A0880008403000007122D
:100C9000831200348316AE012D082E0203186C2E29
:100CA0002B08FA002A08AA0A0319AB0AAF007A082F
:100CB000B000C5002F08C40083120B2583162E0830
:100CC0002C07AF000430C2002F08C3008312E325B5
:100CD00002308316AE074C2E83120034831631087F
:100CE000B40010307602F33E0318AD2E0D3E831291
:100CF000DE2E08308316B500B600AD2E0430831604
:100D0000B5001830B600AD2E0D308316B500083092
:100D1000B600AD2E08308316B5001830B600AD2EE3
:100D200003308316B5000830B600AD2E08308316A8
:100D3000B500B600AD2E14308316B5000830B600ED
:100D4000AD2E08308316B500B600AD2E04308316E4
:100D5000B5001830B600AD2E83163008C5002F0838
:100D6000C40083120B258316B30132083302031823
:100D7000DA2E01303307340784000008B800340845
:100D8000330784000008B9003808BA000230C600F2
:100D90003808C8003908C7008312FE2483163608B5
:100DA000BA003508BB00BC01831248250230831607
:100DB000B307B52E83128A150A12E2280A108A1484
:100DC0000A158207792E7E2EAC2EAC2EAC2E842EE8
:100DD0008A2E962E9B2EA12EA62EAC2E902E8316FA
:100DE00039080739BE007608123C031D212FF83060
:100DF000B9053F30BA05BD013E083D020318212F59
:100E00003A08FA003908B90A0319BA0AC2007A087E
:100E1000C300C5004208C40083120B2504308316AA
:100E2000C200BF30C3008312E32502308316C60020
:100E30004008C8003F08C7008312FE248316BD0A7D
:100E4000FC2EBD013C083D0203184A2F3A08FA0067
:100E50003908B90A0319BA0AC2007A08C300C500E2
:100E60004208C40083120B2583163B08BB0ABB0A49
:100E70008400840A0008C30084030008C200023012
:100E8000C6004308C8004208C7008312FE24831628
:100E9000BD0A222F7608123C031D7E2F3A081F3C04
:100EA0000318552F0430C100572F0830C1003E08E9
:100EB000BC0741083C0203187E2F3A08FA003908A3
:100EC000B90A0319BA0AC2007A08C300C500420869
:100ED000C40083120B2504308316C200BF30C30048
:100EE0008312E32502308316C6004008C8003F087D
:100EF000C7008312FE248316BC0A592F83120034C4
:100F00008316BD0101303C023D020318AA2F3B08A5
:100F1000BB0ABB0A8400840A0008BF0084030008DF
:100F2000BE000230C6003F08C8003E08C70083125A
:100F3000FE24013074078316BE007508BF00031835
:100F4000BF0A3F08C5003E08C40083120B25831664
:100F5000BD0A822F3B088400840A0008BF00840376
:100F60000008BE000230C6003F08C8003E08C700A7
:100F70008312FE24003483162108FD3E0318D92F66
:100F8000033E8312E02F20308316C5000930C400D1
:100F900083120B2509308316C9008312112383168F
:100FA000D92F0B308316C900831211238316D92F32
:100FB00083160630C8008312C8208A150A12882CAE
:100FC0000A148A140A158207CA2FD12FC32F2A08A0
:100FD000FE008A159F2C8A110730A9000130EF000E
:100FE0006B208A150A12542F00308C1A0130F80039
:100FF000003429080C1EFA2F99002908EE06003447
:101000008316B5013108B6000310B20C2F0807395A
:10101000F70030080039FA007708083CB4003408BB
:101020003202031815283208B40012307602FE3E50
:1010300003182C28023E8312C92806308316B700F5
:101040000830B8002C2801308316B7001830B800DB
:101050001730B5002C28831630081F3C031867286A
:10106000FF3A031D37282F08033C03186728300870
:10107000C5002F08C4008A1183120B258A15831618
:10108000B30132083302031866283608B60AB60AD6
:101090008400840A0008BA0084030008B900023002
:1010A000C6003A08C8003908C7008A118312FE2416
:1010B0008A1508308316BA000630BB00BC018A11BD
:1010C000831248258A158316B30A4128C52830089B
:1010D000BA002F08B9003108BB003408BC008A11DF
:1010E0008312EF268A1583163808BA003708BB002A
:1010F0003508BC008A11831248258A1583163408E6
:10110000B2020310340DF700B6070830B3003308FD
:101110003202031CA8287508BA007408B900360802
:10112000BB000830BC008A118312EF268A15831693
:101130003808BA003708BB003508BC008A11831292
:1011400048258A1510308316B6070830B30787285C
:101150000730B205B2080319C5287508BA0074082B
:10116000B9003608BB003208BC008A118312EF2692
:101170008A1583163808BA003708BB003508BC004A
:101180008A11831248258A15831683128A150A123A
:10119000EF280A108A100A1182071D282328103010
:1011A0007602F03E0318D02A103ED12A83162C086E
:1011B000B0002B08AF002D08B1002E08B2008A1134
:1011C00083126E2E8A15D02A83162C08B0002B08A5
:1011D000AF002D08B1002E08B20083120028D02ADB
:1011E00083162C08B0002B08AF002D08B1002E0884
:1011F000B2003108B4000310B20C0130B500083061
:10120000B6000E30B3003008C5002F08C4008A11A4
:1012100083120B258A1583162F080139F700300831
:101220000039FA0077087A04031937293408B40A18
:10123000B40A8400840A0008B80084030008B700D8
:101240000230C6003808C8003708C7008A11831268
:10125000FE248A1583163608BA003508BB00330809
:10126000BC008A11831248258A158316B2033208FE
:10127000013C031883293408B40AB40A8400840AA0
:101280000008B80084030008B7000230C600380820
:10129000C8003708C7008A118312FE248A1501305E
:1012A00074078316B7007508B8000318B80A380821
:1012B000C5003708C4008A1183120B258A158316CE
:1012C0003408B40AB40A8400840A0008B80084030D
:1012D0000008B7000230C6003808C8003708C70049
:1012E0008A118312FE248A1583163608BA0035083F
:1012F000BB003308BC008A11831248258A150230CE
:101300008316B2023729B2080319A6293408B40A91
:10131000B40A8400840A0008B80084030008B700F7
:101320000230C6003808C8003708C7008A11831287
:10133000FE248A1583163608BA003508BB00330828
:10134000BC008A11831248258A1583168312D02A7D
:1013500083162C08B0002B08AF002D08B1002E0812
:10136000B2003108B7000310B20C2F080339B500E2
:10137000043CB40032020318BF293208B400013023
:10138000B8001830B9001730B6003008C5002F0873
:10139000C4008A1183120B258A158316B508031918
:1013A000EB293108BB003408BC008A118312802766
:1013B0008A1583163908BA003808BB003608BC0005
:1013C0008A11831248258A1583163408B202031045
:1013D000340DF700B7070430B30033083202031CA2
:1013E0000A2A3708BB000430BC008A118312802708
:1013F0008A1583163908BA003808BB003608BC00C5
:101400008A11831248258A1508308316B7070430DD
:10141000B307ED290330B2050319252A3208033931
:10142000BA003708BB003A08BC008A118312802733
:101430008A1583163908BA003808BB003608BC0084
:101440008A11831248258A1583168312D02A83169F
:101450002C08B0002B08AF002D08B1002E08B200F8
:101460003108B3000310B20C3008FA002F08AF0A9D
:101470000319B00ABA007A08BB00C5003A08C400D4
:101480008A1183120B258A158316B2080319CE2AF6
:10149000B8013308B30AB30A8400840A0008FA00CA
:1014A00084030008B4007A08B5003808B80A183C6C
:1014B000031CBB2A0230C6003508C8003408C70028
:1014C0008A118312FE248A1508308316C9008A11F6
:1014D000831211238A151E30F700F70B6D2A0000C6
:1014E0000E308316C9008A11831211238A15043025
:1014F0008316C200B630C3008A118312E3258A1511
:10150000831634083602031DBA2A35083702031D34
:10151000BA2A3808BA000330BB008A11831220218E
:101520008A1578088316B800B901380839020318FB
:10153000B92A0230C6003508C8003408C7008A112D
:101540008312FE248A1508308316C9008A1183127B
:1015500011238A151E30F700F70BAC2A00000E305D
:101560008316C9008A11831211238A158316B90ABA
:10157000952ABB2A552AB2033008FA002F08AF0A71
:101580000319B00ABA007A08BB00C5003A08C400C3
:101590008A1183120B258A15442A83168312D02AB6
:1015A00000340A108A140A118207D628D628E428A3
:1015B000E428F028D628D628D628D628D628D62813
:1015C000A829D628D628D02A272A83162108FD3E06
:1015D00003182C2B033E8312302B20308316AB00D4
:1015E0000730AA00A530AC000230AD008A1183128A
:1015F0004A268A1509308316C9008A1183121123DD
:101600008A1508308316C8008A118312C8208A15EB
:10161000FF308316A5040F30A6042030AC0007303D
:10162000AB00A530AD000230AE008312CF20831690
:10163000A10803192C2B0B308316C9008A118312C1
:1016400011238A1508308316C8008A118312C82016
:101650008A1583162C2B831683128A150A123F2CA7
:101660000A148A140A118207ED2A1B2BED2A103066
:101670007602F23E03188A2C0E3E8D2C831620082B
:10168000A1002108F700F708831203194C2B013041
:1016900077020319502B552B02308316A100572BCC
:1016A00003308316A100572B83128316A101210852
:1016B000C9008A11831211238A153F308316CA008C
:1016C000FF30C9008A11831295248A158316A10858
:1016D000031D782BA2012208063C031C782B063040
:1016E000C9008A11831211238A158316A20A6B2B53
:1016F0000130C9008A11831211238A15073083161D
:10170000C9008A11831211238A1508308316C90073
:101710008A11831211238A1508308316C8008A1192
:101720008312C8208A1501308316C9008A118312DA
:1017300011238A1507308316C9008A1183121123D9
:101740008A158A2C83162008A1008A118312692D1C
:101750008A158A2C09308316C9008A118312112335
:101760008A151E308316C8008A118312C8208A1574
:101770008A2C83162008A1002108F700F70883129D
:101780000319C72B013077020319CB2BD02B09305B
:101790008316A300D12B0B308316A300D12B831209
:1017A0008316C9018A11831211238A153F308316CB
:1017B000CA00FF30C9008A11831295248A15831646
:1017C000A2012208063C031CEE2B0630C9008A1138
:1017D000831211238A158316A20AE12B2108023CE9
:1017E0000319082C2308C9008A11831211238A15B2
:1017F00018308316C9008A11831211238A15053007
:101800008316C8008A118312C8208A15312C8316CA
:101810000130C9008A11831211238A1507308316FB
:10182000C9008A11831211238A1508308316C90052
:101830008A11831211238A150D308316C8008A116C
:101840008312C8208A1501308316C9008A118312B9
:1018500011238A1507308316C9008A1183121123B8
:101860008A158A2C83162008A1008A118312AA2DBA
:101870008A158A2C83162008A1008312E52A8A2C57
:1018800083162008A1000230A2001730A3002030E8
:10189000C500C4018A1183120B258A1583162108FD
:1018A000F700F708831203195A2C01307702031945
:1018B000652C712C09308316C9008A1183121123FB
:1018C0008A1508308316A100772C0B308316C900C7
:1018D0008A11831211238A1508308316A100772CF0
:1018E00083121F308316A1000830A200A301210833
:1018F000BA002208BB002308BC008A1183124825C5
:101900008A158A2C83162008A1008A118312BB2F06
:101910008A158A2C8A150A12AA2C0A108A100A150E
:1019200082073E2B3E2BA22BA22BAA2BB92BB92B25
:101930003A2C3E2BB92BB92B402C322C822C280868
:10194000FF3E0318AB2C013EB02C7E088316A0008E
:101950008312372BAB2C871107128A110A12EB2F37
:101960000A108A100A158207A52C2808FF3E0318C2
:10197000C72C013ECC2C83162608AC002508AB00F2
:101980002908AD002A08AE008312CF20C72C87118A
:1019900007128A150A12F22C0A108A100A158207F9
:1019A000BB2C8316A30183122C088316A20083127A
:1019B0002B088316A10083122A088316A000043086
:1019C00083126F02FE0083162308A8002208A700D6
:1019D0002108A6002008A5002D30A9007E08AA0035
:1019E0008312B52C0730A9000130EF008A116B205B
:1019F0008A158A150A125B2F2808FF3E0318102D3E
:101A0000013E152D83162508AB002408AA002808DE
:101A1000AC002908AD008A1183124A268A15102DC0
:101A2000871107128A150A123C2D0A148A100A150A
:101A30008207022D8316A30183122C088316A200AD
:101A400083122B088316A10083122A088316A00094
:101A500083122D08EF0083162308A7002208A60092
:101A60002108A5002008A4002D30A80083126F08CB
:101A70008316A9008312FC2CC430A9000430EF07A0
:101A80008A116B208A158A150A12612F8316AE01FE
:101A900010307602F23E03189A2D0E3E8312C82DA6
:101AA00008308316AC00AD009A2D08308316AC00C8
:101AB000AD009A2D0D308316AC000830AD009A2D84
:101AC00004308316AC001830AD009A2D0130831617
:101AD000AC001830AD001730AE009A2D08308316D8
:101AE000AC001830AD009A2D06308316AC000830DB
:101AF000AD009A2D08308316AC00AD009A2D14303D
:101B00008316AC000830AD009A2D14308316AC005B
:101B10000830AD009A2D04308316AC001830AD00AB
:101B20009A2D01308316AC001830AD001730AE008E
:101B30009A2D83162808C5002708C4008A1183122D
:101B40000B258A158316AB012A082B020318C42D16
:101B50002B08290784000008AF000330C600C80125
:101B60002F08C7008A118312FE248A1583162D08B8
:101B7000BA002C08BB002E08BC008A11831248252D
:101B80008A158316AB0AA42D83128A150A12EB2D2F
:101B90000A148A100A158207502D602D552D662DC6
:101BA000992D5A2D6E2D7A2D7F2D852D8B2D912DD2
:101BB000742D7A2D2808FF3E0318EC2D013EF12DDF
:101BC00083162408A8002308A7002508A9002608D2
:101BD000AA008312462DEC2D871107128A150A12CE
:101BE0000C2E0A148A100A158207E02D2B08831682
:101BF000A10083122A088316A000033083126F020B
:101C0000FE0083162108A4002008A3002C30A500A4
:101C10007E08A6008312DA2D0730A9000130EF00FC
:101C20008A116B208A158A150A12672F2808FF3E31
:101C300003184D2E013E522E83162308A7002208BA
:101C4000A6002408A8002508A900AA0129082A023C
:101C500003184B2E2708FA002608A60A0319A70A1C
:101C6000AD007A08AE00C5002D08C4008A118312A9
:101C70000B258A1505308316C200AB30C3008A11CC
:101C80008312E3258A1583162A08280784002B0867
:101C90008000AA0A262E83124D2E871107128A155C
:101CA0000A126E2E0A108A140A1582071C2E2B089F
:101CB0008316A10083122A088316A00083122C0821
:101CC000EF0083162108A3002008A2002C30A400F6
:101CD00083126F088316A5008312162EE230A90026
:101CE0000330EF078A116B208A158A150A126D2FAF
:101CF0008A114B208A15D030A900AA01AB01AC0192
:101D0000AD010530EF008A116B208A158A150A1281
:101D1000732F8A116F228A15D030A9000130AA00D2
:101D2000AB01AC01AD010530EF008A116B208A15C3
:101D30008A150A12792F0130FD008316A20129307D
:101D4000A300A208031DED2E8A11831254208A15C8
:101D50007808FE007E08043C0319B42E8A11542032
:101D60008A157808FE00AA2E8A1154208A15780850
:101D7000EF008316A100A00183126F0883162002D2
:101D80000318D42E2308A4008A11831254208A1524
:101D90008316240884007808800023088400000843
:101DA000A106A30AA00ABC2E8A11831254208A1508
:101DB00078088316A106031DE62E0130A200063026
:101DC00083120C1EE12E9900EB2E83160530831230
:101DD0000C1EE82E99008316A12E83122908103CB0
:101DE000031DF62E8A11B4208A157B2F2908113C79
:101DF000031DFE2E8A11DD288A157B2F2908123C2F
:101E0000031D062F8A1147298A157B2F2908143CA8
:101E1000031D0E2F8A11D6298A157B2F2908153C00
:101E2000031D162F8A11A2218A157B2F2908173C22
:101E3000031D1E2F8A11F0298A157B2F2908183CB3
:101E4000031D262F8A11322A8A157B2F29081A3C56
:101E5000031D2E2F8A115B2A8A157B2F29081B3C14
:101E6000031D362F8A11652A8A157B2F2908413CCC
:101E7000031D3E2F8A11B22A8A157B2F2908403C68
:101E8000031D462F8A11C42A8A157B2F2908473C37
:101E9000031D4E2F8A11052B8A157B2F2908433CE1
:101EA000031D562F8A11E72F8A157B2F2908423CE4
:101EB000031D5C2FD12C7B2F2908443C031D622F6E
:101EC0001A2D7B2F2908453C031D682FF62D7B2FEB
:101ED0002908463C031D6E2F572E7B2F2908503CA6
:101EE000031D742F782E7B2F2908513C031D7A2F58
:101EF000892E7B2FFD017D08F8008A150A16972C84
:101F000083164B1464008312071E9A2F64008316F5
:101F10004A08CA03003A031D922F4B1083129A2FCE
:101F2000992F83164D30F700F70B942F0000000017
:101F30008312842F003083164B180130F80083126F
:101F400000340830F7000718A32F8316BA01F717DB
:101F5000B92FF713B92F0310831207180314831630
:101F6000BA0C7717B92F7713F70BAB2F3A08F80095
:101F7000C62F7930F71B2130F800F80BBD2F000079
:101F80000000F71BA92F771BB32FAB2F83128A11E9
:101F90000A16632908300C1ECB2F990083163608C9
:101FA00083120C1ED12F9900003407100830F8005E
:101FB000000000000000F817EE2FF8138316B70C8E
:101FC000831203180714031C07107817EE2F7813D9
:101FD000F80BDE2F000000000000071479308400A9
:101FE000840BF02F00000000F81BDD2F781BE72F7B
:101FF0008A110A16FD2983162908F8008312003475
:102000008316420DC300C30DC30DF830C305071678
:10201000FF30CA000A128A15831280270A168A1115
:102020008316C501C40145087102031C2528031D40
:102030001D2844087002031C25280230F700F70B06
:102040001F28C40A0319C50A13288312871583168B
:10205000C501C40145087102031C3D28031D342835
:1020600044087002031C3D280630F700F70B3628A1
:102070000000C40A0319C50A2A288312071A422835
:102080000310432803148316C60DC70DC80D07128D
:10209000831207128316420B53280310BE0D031C34
:1020A0005328071668284208023C031D5E280310C7
:1020B000BE0DBF0D031C5E28071668284208033CAE
:1020C000031D68280310BE0DBF0DC00D03180716B1
:1020D000831287118316C501C40145087102031CD0
:1020E0008028031D772844087002031C80280630CE
:1020F000F700F70B79280000C40A0319C50A6D28F8
:102100000716C30B252807164608F7004708F800EE
:102110004808F9004908FA0083120034FF3083169A
:10212000B400B500B600B701CA010A128A158312BD
:1021300080270A168A11F8080319BE282808FF3ECE
:102140000318BE28013EC9288316C101C0014030D2
:10215000BF00BE010230C2008312002078081F3980
:10216000FA007708F8007A08F9008316B701B6017B
:102170007908B5007808B4008312BE2883163408A5
:10218000F7003508F8003608F9003708FA0083121E
:1021900000340A108A100A118207A428FF3083161F
:1021A000B000B100B200B301CA010A128A1583124D
:1021B00080270A168A11F808031931292808FF3EDA
:1021C00003183129013E3C2A83162C08B5002B0840
:1021D000B4002C08B7002B08B600FF30B800B900D7
:1021E0003608F70037081F39FA003608BA007A08AF
:1021F000C038BB00BC01BD013D08C1003C08C000A7
:102200003B08BF003608BE000230C2008312002027
:102210008316CA010A128A15831280270A168A11A8
:10222000F808031924298316C101C0014030BF00FA
:10223000BE010230C2008312002077088316B80066
:1022400078081F39B900831283163808F800390856
:10225000F900B301B2017908B1007808B000831227
:1022600031298316AF080319142A34103418142A9C
:10227000CA010A128A15831280270A168A11F808E1
:10228000031944298316142AB5308316B60037146F
:10229000B710861083128614831607147C1C5529E8
:1022A00036088400013080009029B7189029640016
:1022B000831207186D29831636088400B9000A12A4
:1022C0008A158312A12F0A168A11831639088400F1
:1022D00078088000B7148F2983120A12F4270A168F
:1022E000F80803197F290A1254200A167808023CBC
:1022F000031D7E298316B714371083128E29831687
:10230000CA010A128A15831280270A168A11F80850
:1023100003198E298316B714371083128316552993
:10232000003037180130F800F8080319102A350872
:10233000F70001307702831203199F29052A013023
:102340008316B6000A128A158312CA270A168A1142
:10235000B5308316B6003714B710B718EB29CA0189
:102360000A128A15831280270A168A11F80803199F
:10237000BB298316EB290A12F4270A16F808031959
:10238000E92983163608B8000A12831254200A1667
:102390008316380884007808800036088400000816
:1023A000083C031DE0293608B8000A1283125420A5
:1023B0000A1683163808840078088000B714E829C4
:1023C000360884000008023C031DE829B7143710C2
:1023D00083128316AD29003037180130F800F80851
:1023E0000319012A7C103508B60086140710360838
:1023F000B7000A128A158312D52F0A168A11042AE9
:1024000083167C14341483120E2A83163508B60002
:102410000A128A158312CA270A168A11122A8316EB
:102420003414831283163629300F1D2A310F1D2ACA
:10243000320F1D2AB3080319272A300F322A310F11
:10244000322AB208031D322AB308031D322A83122E
:102450008E207A088316B3007908B2007808B1009C
:102460007708B0003008F7003108F8003208F900AA
:102470003308FA00831200340A108A140A11820702
:10248000E4280A124B200A1687150A126F220A1630
:102490000230F700F70B4A2A000000008711FF30D6
:1024A0008316CA000A128A15831280270A168A1117
:1024B0008316AE01AD01AC01AB01AF018312CE209A
:1024C0000A124B200A1687150A126F220A160230CA
:1024D000F700F70B692A0000000087118316C1017D
:1024E000C0014030BF00BE010230C2008312002094
:1024F00078081F39FA007708F8007A08F9000034E4
:102500008316A901AA01F1017330F000FF30CA005F
:102510000A128A15831280270A168A11F8080319ED
:10252000F22A8316C101C0011030BF00BE01023083
:10253000C20083120020831607168312071A9E2AF0
:102540008316AA01A90183128715F3010130F20055
:10255000071AB32AF20A0319F30A7208730403195B
:10256000B32A6400A82A071ABE2AF20A0319F30A3A
:10257000720873040319BE2A6400B32A8312071E6B
:10258000D02A8316A90A0319AA0A29082A040319BA
:10259000D02A12306400FF3E031DCA2A0000BE2A62
:1025A00083128711720873040319ED2A8316290810
:1025B0002A04031DDD2A8312ED2A2A0CF100290CBE
:1025C000F000F10CF00CF10CF00CF10CF00CF10C33
:1025D000F00C0730F105F12A8312F1017330F0009D
:1025E0008316831283162908F8002A08F90083123B
:1025F0000034831605118312051583168512831284
:10260000851683168610831286142808FF3E031849
:10261000162B013E372B412241228316A801A70128
:102620007908A6007808A5008312162B8022FF30B7
:102630008316CA000A128A15831280270A168A1185
:10264000F808031D2A2B8316A801FF30A700A60057
:10265000A500831283162508F7002608F80027082E
:10266000F9002808FA0083128A110A16412B0A146D
:102670008A140A1182070B2BA0308316A400831240
:10268000F92A7A088316A3007908A2007808A10025
:102690007708A000D0308312A9008316CA010A125D
:1026A0008A15831280270A168A11F80803195A2BF3
:1026B00000305B2B0130AA0083162408A40A840092
:1026C00000088312AB0083162408A40A84000008C3
:1026D0008312AC0083162408840000088312AD0026
:1026E0000530EF000A126B200A168A150A16CB2B4A
:1026F0008316A801FF30A700A600A500CA010A1290
:102700008A15831280270A168A11F808031DB82B30
:1027100087151E30F700F70B8B2B00008711280858
:10272000FF3E0318AF2B013EC52B8316C101C0012C
:102730004030BF00BE010230C20083120020780882
:102740001F39FA007708F8007A08F9008316A80103
:10275000A7017908A6007808A5008312AF2BFF30E7
:102760008316CA000A128A15831280270A168A1154
:1027700083162508F7002608F8002708F90028081E
:10278000FA0083128A110A16CF2B0A148A140A112E
:102790008207952BA0308316A4008312782B7A0829
:1027A0008316A3007908A2007808A1007708A0008A
:1027B000D0308312A9008316CA010A128A15831227
:1027C00080270A168A11F8080319E82B0030E92B34
:1027D0000130AA0083162408A40A8400000883128A
:1027E000AB0083162408A40A840000088312AC00FE
:1027F00083162408840000088312AD000530EF0022
:102800000A126B200A168A150A16D32B8316251472
:10281000A030A40083126F08053C031D1B2C2D085B
:102820000139003A031D182C831625101A2C831227
:102830008316251483128316A90183122C0883168C
:10284000A80083122B088316A70083122A08831678
:10285000A600003025180130AA002908AE0028087B
:10286000AD002708AC002608AB002A08AF00831291
:10287000CE207A088316A3007908A2007808A10068
:102880007708A000D0308312A9008316CA010A126B
:102890008A15831280270A168A11F8080319522C08
:1028A0000030532C0130AA0083162408A40A8400A7
:1028B00000088312AB0083162408A40A84000008D1
:1028C0008312AC0083162408840000088312AD0034
:1028D0000530EF000A126B200A168A150A16DB2B48
:1028E000FF308316CA000A128A15831280270A163F
:1028F0008A11F8080319A62C2808FF3E0318A62CF5
:10290000013EC62C8316C101C001FF30BF00BE00CE
:102910000230C200831200208316C101C001403082
:10292000BF00BE010230C2008312002078081F39A8
:10293000FA007708F8007A08F9008316A801A701C1
:102940007908A6007808A5008312A62CFF3083160C
:10295000CA000A128A15831280270A168A11F808FB
:10296000031DB92C8316A801FF30A700A600A500FF
:10297000831283162508F7002608F8002708F900B7
:102980002808FA0083128A110A16052F0A108A10E5
:102990000A158207822C03300C1ECC2C990083165A
:1029A000260883120C1ED22C990083162608831247
:1029B000EE0000348316A901FF30CA000A128A15FE
:1029C000831280270A168A11F8080319F42C83163B
:1029D000C101C001BF01BE010130C200831200204D
:1029E00077088316A900831283162908F80083123A
:1029F000003465200A168A150A166D28FF3FFF3F2E
:102A000084011F308305073083169F000230990030
:102A100022309800903083129800A001A10110305C
:102A2000A2003030A3008A30A400A501A6012D30F9
:102A3000A700FF30EF00EF106F08831687008312A6
:102A40008714023083169900223098009030831248
:102A5000980002308316990022309800903083123B
:102A600098000F30F70007308101813084000008A2
:102A7000F0390738800064000008F03977048000DE
:102A8000A32564009626412D63000C1E452D990058
:102A90007A2D0530F6007608063C03197A2D8C1A3B
:102AA000532D64004F2D8C1E532D1A088316A00041
:102AB0008312981C612D1A088316A0008312181225
:102AC000181683162008F800831200342808073CE3
:102AD000031D6F2D07300C1E6B2D9900A22D0530A4
:102AE000FC007C08063C0319A22D7C08053C031D54
:102AF0009E2D2830FE006E08F60004300C1E7E2D40
:102B000099006E080C1E822D9900FD016E087D0251
:102B100003189A2D7E08840000088316A0008312F3
:102B20000C1E902D99007E0884000008F606FE0A0F
:102B3000FD0A862D76080C1E9B2D99004F257808DE
:102B4000FC00712D0034B130A8000130EE00662584
:102B50000034F3012830F400F308031DE42D4F2561
:102B60007808F0007008043C0319BA2D4F25780846
:102B7000F000B22D4F257808EE006E08F200F1014A
:102B80006E0871020318D22D7408F5004F257508E0
:102B9000840078088000740884000008F206F40AB3
:102BA000F10AC02D4F257808F206F208031DDF2D2B
:102BB0000130F30006300C1EDB2D9900E32D0530AB
:102BC0000C1EE02D9900AC2D003403306E02003A4B
:102BD0000319502EF1012A08F0007008F1002908AD
:102BE000F0002B30F5000330F4006E087402031877
:102BF000502E7508F50A84000008FA01F2007A08E0
:102C0000F3007508F50A84000008F600F300710867
:102C1000143C03180F2E7108163C03184A2E710835
:102C20001F3C031C4A2EF108031D292E7008033C8B
:102C3000031C292E0310700DF900710DFA0079089C
:102C4000203E8400840A7308800084037208800098
:102C50004A2E700803178D0071088F0072088C00CF
:102C600073088E0083168C170C15831203130B0840
:102C7000F8008B138316031755308D00AA308D0092
:102C80008C14000000008C18432E0C11780883125D
:102C900003138B04F00A0319F10A0230F407F52D2F
:102CA0000730A8000130EE0066250034F0017008FE
:102CB000033C031C8C2EF2017008F1000310700D10
:102CC000F700203E8400840A0008F4008403000812
:102CD000F300700803178D0072088F0073088C00D2
:102CE00074088E0083168C170C15831203130B08BF
:102CF000F8008B138316031755308D00AA308D0012
:102D00008C14000000008C18832E0C11780883129C
:102D100003138B04F00A572E8C2E00342808A900C8
:102D2000FF30A8000230EE0066250034A9252808EF
:102D3000F700313077020319A62E323077020319DB
:102D4000A82E333077020319AA2EAC2EA325AE2E5F
:102D5000E525AE2E5626AE2E8E26AE2E0034FF3F33
:102D6000FF3FFF3FFF3FFF3FFF3FFF3FFF3FFF3F73
:102D7000FF3FFF3FFF3FFF3FFF3FFF3FFF3FFF3F63
:102D8000FF3FFF3FFF3FFF3FFF3FFF3FFF3FFF3F53
:102D9000FF3FFF3FFF3FFF3FFF3FFF3FFF3FFF3F43
:102DA000FF3FFF3FFF3FFF3FFF3FFF3FFF3FFF3F33
:102DB000FF3FFF3FFF3FFF3FFF3FFF3FFF3FFF3F23
:102DC000FF3FFF3FFF3FFF3FFF3FFF3FFF3FFF3F13
:102DD000FF3FFF3FFF3FFF3FFF3FFF3FFF3FFF3F03
:102DE000FF3FFF3FFF3FFF3FFF3FFF3FFF3FFF3FF3
:102DF000FF3FFF3FFF3FFF3FFF3FFF3FFF3FFF3FE3
:102E0000A0308316A4008312702C7A088316A300C6
:102E10007908A2007808A1007708A000D0308312BA
:102E2000A9008316CA010A128A15831280270A167E
:102E30008A11F80803191E2F00301F2F0130AA0035
:102E400083162408A40A840000088312AB008316AA
:102E50002408A40A840000088312AC008316240806
:102E6000840000088312AD000530EF000A126B20C9
:102E70000A168A150A16E32BA0308316A4008312C3
:102E80008E207A088316A3007908A2007808A10092
:102E90007708A000D0308312A9008316CA010A1255
:102EA0008A15831280270A168A11F80803195A2FE7
:102EB00000305B2F0130AA0083162408A40A840086
:102EC00000088312AB0083162408A40A84000008BB
:102ED0008312AC0083162408840000088312AD001E
:102EE0000530EF000A126B200A168A150A16EB2B22
:102EF0006E080C1E792F99000A1254200A167808C1
:102F0000063C031D7C2F00342B088316A20083127D
:102F10002A088316A1000330A00083126F088316CD
:102F200020020318EA2F2208FA002108A10A031937
:102F3000A20AA3007A08A400293020078400000810
:102F4000A5002408A7002308A6002508A800FF3034
:102F5000CA000A128A15831280270A168A11F808F5
:102F60000319E72F83162608F70027080F39FA0000
:102F70002608A9007A085038AA00AB01AC012C0839
:102F8000C1002B08C0002A08BF002608BE0002307E
:102F9000C20083120020FF308316CA000A128A156D
:102FA000831280270A168A1183162808A900603028
:102FB000AA00AB01AC012C08C1002B08C0002A08F4
:102FC000BF002808BE000230C20083120020831612
:102FD000A00A8D2F07308312A9000130EF000A12DA
:102FE0006B200A168A150A16F92B0A1600342A08CD
:102FF000F80083120034FF3FFF3FFF3FFF3FFF3FDA
:1030000029308316A20083122B088316A100831295
:103010002A088316A00083122C088316A40003300C
:103020002407A500A6008A118312CB248A158316D3
:1030300022088400E03080000A128A118312F927E6
:103040000A168A1583162208840083122A08800033
:103050000A128A11F9270A168A1583162208840093
:1030600083122B0880000A128A11F9270A168A1582
:1030700083162208A5002108A7002008A600FF301B
:10308000CA000A12831280270A16F80803196A2850
:1030900083162608F70027080F39FA002608A9002A
:1030A0007A084038AA00AB01AC012C08C1002B08FB
:1030B000C0002A08BF002608BE000230C2008A11E4
:1030C000831200208A158A11DA248A15780883165B
:1030D000A8008312FF308316CA000A1283128027C9
:1030E0000A16F808031D7828FF308316A8008312FB
:1030F00083162808F80025088400780880000A1242
:103100008A118312F9270A168A1501308316A30043
:10311000240823020318A0282208A5008A1183127C
:10312000DA248A15831625088400780880000A129C
:103130008A118312F9270A168A158316A30A88288A
:103140008A11831278278A158A150A16F22B83169C
:103150002C08AD002030AE00AF01B0013008C10036
:103160002F08C0002E08BF002D08BE000230C2008C
:103170008A11831200208A158316C101C0014030D4
:10318000BF00BE010230C2008A11831200208A15DE
:1031900078088316AF007708AE002F08FA01F80010
:1031A000831200348316AA01FF30CA000A12831268
:1031B00080270A16F8080319ED282808FF3E03188F
:1031C000ED28013EF42883162808AC008312A720BE
:1031D00078088316AA008312ED2883162A08F800BF
:1031E00083128A150A1647290A108A100A118207C3
:1031F000E32829308316A20083122B088316A1002E
:1032000083122A088316A00083122C088316A400B8
:1032100003302407A500A6008A118312CB248A1547
:10322000831622088400E23080000A128A11831279
:10323000F9270A168A1583162208840083122A08A1
:1032400080000A128A11F9270A168A1583162208A5
:10325000840083122B0880000A128A11F9270A16AB
:103260008A158316A301240823020318552922086E
:10327000A5002108FA002008A00A0319A10AA60047
:103280007A08A700A9002608A8008312D22883166E
:1032900025088400780880000A128A118312F92711
:1032A0000A168A158316A30A33298A1183127827EE
:1032B0008A158A150A16002CFF308316CA000A12D6
:1032C000831280270A16F8080319A8292808FF3E48
:1032D0000318A829013EAB2983162308A700250857
:1032E000A8002608A900AA0129082A020318A6296D
:1032F0002A082707AB00AC008312A72083162808F2
:103300002A0784000008AB00AC00FF30CA000A1294
:10331000831280270A16F8080319A32983162C089C
:10332000AD003030AE00AF01B0013008C1002F0851
:10333000C0002E08BF002C08BE000230C2008A1157
:10334000831200208A158316AA0A74298312A829D9
:103350008A150A16C6290A148A100A1182076C29CE
:103360002B088316A10083122A088316A0000330BD
:1033700083126F028316A2002108A4002008A30074
:103380002C30A5002208A60083125C290730A90072
:103390000130EF000A128A116B200A168A158A156D
:1033A0000A16062CFF308316CA000A1283128027E1
:1033B0000A16F80803192E2A2808FF3E03182E2A99
:1033C000013E312A83162608AC002508AB002908E7
:1033D000AD002A08AE002B08B0002C08B100083060
:1033E000B200B3013308C1003208C0002C08BF008E
:1033F0002B08BE000330C2008A11831200208A15F8
:103400008316C1010930C000BF01BE010330C200F4
:103410008A11831200208A158316AF012E082F020D
:1034200003182C2A2D08AD0AAD0AB000C1010930DD
:10343000C000BF01BE010330C2008A118312002008
:103440008A1583163008840077088000840A78087B
:1034500080000230AF070E2A83122E2A8A150A1620
:10346000582A0A108A140A118207E2298316A40135
:1034700083122C088316A30083122B088316A20044
:1034800083122A088316A10083122D08EF008316E9
:103490002408A8002308A7002208A6002108A500E8
:1034A0002D30A90083126F088316AA008312D22937
:1034B000C430A9000430EF070A128A116B200A16E3
:1034C0008A158A150A160C2CFF308316CA000A12B8
:1034D000831280270A16F8080319BB2A2808FF3E22
:1034E0000318BB2A013EBE2A83162708AD00260812
:1034F000AC002A08AE002B08AF002C08B1002D0844
:10350000B2000830B300B4013408C1003308C00071
:103510002D08BF002C08BE000330C2008A118312A0
:1035200000208A158316B0012F0830020318B92A2B
:103530002E08AE0AAE0A8400840A0008FA0084034A
:103540000008B1007A08B2000A30B300B4013408B0
:10355000C1003308C0003208BF003108BE0003308C
:10356000C2008A11831200208A1502308316B00728
:10357000942A8312BB2A8A150A16E42A0A108A148E
:103580000A118207742A8316A40183122C08831659
:10359000A30083122B088316A20083122A08831625
:1035A000A100043083126F028316A5002408A9002D
:1035B0002308A8002208A7002108A6002D30AA0091
:1035C0002508AB008312642A0730A9000130EF0000
:1035D0000A128A116B200A168A158A150A16122CED
:1035E0002A308316A00097308312A9008316200882
:1035F000A1008A11831280228A1583162108840073
:10360000840A7908800084037808800003308312DC
:10361000EF000A128A116B200A168A158A150A16FB
:10362000182C2A308316A00083122C08EF00831672
:1036300020088400840A0008A20084030008A10076
:103640002208A4002108A3002C30A50083126F08D3
:103650008316A600E6308312A9000330EF070A1292
:103660008A116B200A168A158A150A161E2C2A3012
:103670008316A00020088400840A0008A2008403A6
:103680000008A100033083126F028316A3002208F2
:10369000A5002108A4002C30A6002308A7000730AD
:1036A0008312A9000130EF000A128A116B200A165A
:1036B0008A158A150A16242C8316A0012008033CBB
:1036C000031CAE2BA2012008A1000310200DF7005F
:1036D000A300230A0A128A11831235200A168A15BA
:1036E000FA00831623080A128A11831235200A165B
:1036F0008A158316A4007A08A500210883120317EF
:103700008D00831603132208831203178F0083167C
:1037100003132408831203178C0083160313250850
:10372000831203178E0083168C170C158312031354
:103730000B08F8008B138316031755308D00AA3041
:103740008D008C14000000008C18A42B0C1178083C
:10375000831203138B048316A00A5E2B8A01831243
:1037600082018A150A162A2C2908AA00FF30A9000E
:103770000230EF000A128A116B200A168A158A1588
:103780000A162C2CFE08031D2C2C2908523C031D64
:10379000CD2B8A113C2B8A152C2C2908533C031D58
:1037A000D52B8A11CA2B8A152C2C2908543C031DB1
:1037B000DD2B8A11062C8A152C2C2908553C031D5B
:1037C000E52B8A11002F8A152C2C2908563C031D45
:1037D000ED2B8A113C2F8A152C2C2908603C031DE7
:1037E000F32B00282C2C2908613C031DFB2B8A118C
:1037F000842F8A152C2C2908623C031D012CF928E2
:103800002C2C2908633C031D072CB0292C2C2908DB
:10381000653C031D0D2C362A2C2C2908643C031D05
:10382000132CC32A2C2C2908663C031D192CF02AC2
:103830002C2C2908673C031D1F2C112B2C2C29082C
:10384000683C031D252C372B2C2C2908313C031DEB
:103850002B2C5C2B2C2CB42B8A150A169C2C840147
:103860001F308305073083169F00023099002230F5
:10387000980090308312980002308316990022300D
:1038800098009030831298000230831699002230FD
:1038900098009030831298000230831699002230ED
:1038A00098009030831298000230831699002230DD
:1038B00098009030831298007330F000F1017C1072
:1038C00007140714993083168700103086000B30D8
:1038D0008500B530831290008F018E0183160C1481
:1038E000C03083128B040F30F70007308101813024
:1038F00084000008F0390738800064000008F039BF
:10390000770480000A128A114B200A168A150A12BF
:103910008A11B4200A168A150B138B138B1B8D2C5E
:1039200083160C108312061564000A129B2E0A16C9
:103930007808FD00FE00C22B942C63008D008C14CF
:10394000000000008C18A22C0C11780883120313BD
:103950008B04FE0A5B2C8A01820100342808A9002E
:10396000FF30A8000230EE000A128A1165200A1604
:103970008A15003484011F308305073083169F00A9
:103980000230990022309800903083129800023063
:1039900083169900223098009030831298000230EC
:1039A00083169900223098009030831298000230DC
:1039B00083169900223098009030831298000230CC
:1039C000831699002230980090308312980073304B
:1039D000F000F1017D100714071499308316870059
:1039E000103086000B308500B530831290008F01B7
:1039F0008E0183160C14C03083128B040F30F70035
:103A000007308101813084000008F03907388000D8
:103A100064000008F039770480000A128A114B20F4
:103A20000A168A150A128A11AE200A168A158316FA
:103A3000A2012830A300A208031D712D0A128A11C9
:103A400083124E200A168A157808FE007E08043C70
:103A50000319322D0A128A114E200A168A15780887
:103A6000FE00262D0A128A114E200A168A157808A1
:103A7000EE008316A100A00183126E0883162002B7
:103A80000318562D2308A4000A128A1183124E200F
:103A90000A168A15831624088400780880002308F3
:103AA00084000008A106A30AA00A3C2D0A128A116C
:103AB00083124E200A168A1578088316A106031D64
:103AC0006A2D0130A200063083120C1E652D99006C
:103AD0006F2D8316053083120C1E6C2D99008316F2
:103AE0001B2D83122808F700103028020319E12D3E
:103AF000113077020319E72D123077020319ED2DEB
:103B0000143077020319F32D153077020319F92DBC
:103B1000173077020319FF2D183077020319052E8D
:103B20004130770203190B2E403077020319112E12
:103B3000473077020319172E4330770203191D2EE1
:103B4000423077020319212E443077020319252EC3
:103B5000453077020319292E4630770203192D2E9E
:103B6000503077020319312E513077020319372E66
:103B70005230770203193B2E5330770203193F2E40
:103B8000543077020319412E553077020319432E22
:103B9000563077020319452E603077020319472EFD
:103BA000613077020319492E6230770203194B2ED8
:103BB0006330770203194D2E3130770203194F2EEF
:103BC000512E0A128A11AE200A168A15522E0A1296
:103BD0008A11D7200A168A15522E0A128A113F21FD
:103BE0000A168A15522E0A128A11CC210A168A1533
:103BF000522E0A128A1198210A168A15522E0A127A
:103C00008A11E4210A168A15522E0A128A112422D8
:103C10000A168A15522E0A128A1184220A168A1549
:103C2000522E0A128A1194220A168A15522E0A124C
:103C30008A11C4220A168A15522E0A122B220A163B
:103C4000522E0A1222230A16522E0A128B240A1608
:103C5000522E0A120B260A16522E8A113E208A155F
:103C6000522E0A128A11F1270A168A15522E0A12AA
:103C7000C9270A16522E8A1100278A15522E0020B3
:103C8000522E8E20522ED920522E7D21522E3A2293
:103C9000522EBE22522E5223522EE123522E5A244D
:103CA000522EAE240B138B138B1B532E83160C102A
:103CB0008312061564008316A2012830A300A2080F
:103CC000031DB52E0A128A1183124E200A168A1578
:103CD0007808FE007E08043C0319762E0A128A1129
:103CE0004E200A168A157808FE006A2E0A128A11DA
:103CF0004E200A168A157808EE008316A100A0014E
:103D000083126E088316200203189A2E2308A4003B
:103D10000A128A1183124E200A168A158316240865
:103D2000840078088000230884000008A106A30A04
:103D3000A00A802E0A128A1183124E200A168A15B2
:103D400078088316A106031DAE2E0130A2000630AE
:103D500083120C1EA92E9900B32E831605308312F0
:103D60000C1EB02E990083165F2E83122808F700D0
:103D7000103028020319252F1130770203192B2F39
:103D8000123077020319312F143077020319372FBD
:103D90001530770203193D2F173077020319432F8F
:103DA000183077020319492F4130770203194F2F3A
:103DB000403077020319552F4730770203195B2FE4
:103DC000433077020319612F423077020319652FC0
:103DD000443077020319692F4530770203196D2F9C
:103DE000463077020319712F503077020319752F6F
:103DF0005130770203197B2F5230770203197F2F3E
:103E0000533077020319832F543077020319852F1B
:103E1000553077020319872F563077020319892FFF
:103E20006030770203198B2F6130770203198D2FD1
:103E30006230770203198F2F633077020319912FB5
:103E4000313077020319932F952F0A128A11AE2071
:103E50000A168A15962F0A128A11D7200A168A1571
:103E6000962F0A128A113F210A168A15962F0A12D6
:103E70008A11CC210A168A15962F0A128A119821C6
:103E80000A168A15962F0A128A11E4210A168A1533
:103E9000962F0A128A1124220A168A15962F0A12C0
:103EA0008A1184220A168A15962F0A128A119422E0
:103EB0000A168A15962F0A128A11C4220A168A1522
:103EC000962F0A122B220A16962F0A1222230A165E
:103ED000962F0A128B240A16962F0A120B260A1600
:103EE000962F8A113E208A15962F0A128A11F127E1
:103EF0000A168A15962F0A12C9270A16962F8A11B2
:103F000000278A15962F0020962F8E20962FD920D5
:103F1000962F7D21962F3A22962FBE22962F52233E
:103F2000962FE123962F5A24962FAE245A2E630003
:103F3000220803178C000313210803178E00831631
:103F400003178C170C158B1355308D00AA308D007C
:103F50008C140000FF3EFF3EFF3EFF3EFF3EFF3E53
:103F6000FF3EFF3EFF3EFF3EFF3EFF3EFF3EFF3E69
:103F7000FF3EFF3EFF3EFF3E0C118C1383016400A9
:103F80000D1EBF2F0D1283168101831269080317BE
:103F90008D000313680803178F00DC2783120317B3
:103FA0000C080313A20003170E080313A100080056
:103FB000E90A0319E80A0800831603178C170C1482
:103FC0000000FF3EFF3E8C138301080021081F39CB
:103FD000E8001F3A031968122208E900C627462E96
:103FE00068081E391E3A0319FC2F6808031DFB2FB1
:103FF0006908C039031D8B27D827462EFF3FFF3F96
:104200000200FF00FF00FF00FF00FF00FF00FF00B3
:10421000FF00FF00FF00FF00FF00FF00FF00FF00A6
:10422000FF00FF00FF00FF00FF00FF00FF00FF0096
:10423000FF00FF00FF00FF00FF00FF00FF00FF0086
:10424000FF00FF00FF00FF00FF00FF00FF00FF0076
:10425000FF00FF00FF00FF00FF00FF00FF00FF0066
:10426000FF00FF00FF00FF00FF00FF00FF00FF0056
:10427000FF00FF00FF00FF00FF00FF00FF00FF0046
:10428000FF00FF00FF00FF00FF00FF00FF00FF0036
:10429000FF00FF00FF00FF00FF00FF00FF00FF0026
:1042A000FF00FF00FF00FF00FF00FF00FF00FF0016
:1042B000FF00FF00FF00FF00FF00FF00FF00FF0006
:1042C000FF00FF00FF00FF00FF00FF00FF00FF00F6
:1042D000FF00FF00FF00FF00FF00FF00FF00FF00E6
:1042E000FF00FF00FF00FF00FF00FF00FF00FF00D6
:1042F000FF00FF00FF00FF00FF00FF00FF00FF00C6
:10430000FF00FF00FF00FF00FF00FF00FF00FF00B5
:10431000FF00FF00FF00FF00FF00FF00FF00FF00A5
:10432000FF00FF00FF00FF00FF00FF00FF00FF0095
:10433000FF00FF00FF00FF00FF00FF00FF00FF0085
:10434000FF00FF00FF00FF00FF00FF00FF00FF0075
:10435000FF00FF00FF00FF00FF00FF00FF00FF0065
:10436000FF00FF00FF00FF00FF00FF00FF00FF0055
:10437000FF00FF00FF00FF00FF00FF00FF00FF0045
:10438000FF00FF00FF00FF00FF00FF00FF00FF0035
:10439000FF00FF00FF00FF00FF00FF00FF00FF0025
:1043A000FF00FF00FF00FF00FF00FF00FF00FF0015
:1043B000FF00FF00FF00FF00FF00FF00FF00FF0005
:1043C000FF00FF00FF00FF00FF00FF00FF00FF00F5
:1043D000FF00FF00FF00FF00FF00FF00FF00FF00E5
:1043E000FF00FF00FF00FF00FF00FF00FF00FF00D5
:1043F000FF00FF00FF00FF00FF00FF00FF00FF00C5
:02400E003D3F34
:00000001FF
